:1000000000308A00FD2D0000A60003088312A8001E
:100010000A08A7008A118B1C22288B10A914AB0A8E
:10002000031086180314AC0DAD0DAE0D291E222849
:10003000320803192228B203B10CB00CAF0C061120
:100040000318061527088A0028088300A60E260E26
:10005000090000000000000000000130831630029B
:1000600003193428831237288312051238280516FD
:100070000034B310B311AC01AD01AE01AB01BF014F
:1000800000343310B501B601B201FF30B800A90148
:10009000AF01B001B10139208316A70183120430EA
:1000A00083162702031C56288312612883123930D5
:1000B000831627078400800183128316A70A831200
:1000C0004F2807088316A800A80E0F30A805A80916
:1000D00028080F398312A1002108B4008130840060
:1000E00000170B168B108A111F2E053090008F0100
:1000F0008E01101483160C1083120C108A11202EFE
:10010000A001A01D8B2807308101813084000008E8
:10011000C0390F3880006400813084000008C03985
:1001200020048000833081000B118A11212E831658
:10013000B5018312831634083502031CA1288312EB
:10014000B7288312640014308316B60083128330FC
:1001500081000B110B1DAA288316B60BB028B228FC
:100160008312A72883128316B50A83129A280034B3
:100170008316B308031DBE288312C22883120714F6
:100180000616C4280710061214308316B400831212
:10019000972000348316AD08031DD0288312D3287E
:1001A00083120715D428071101308316B400831277
:1001B00097200034013083162D020319E1288312A1
:1001C000E42883128616E52886128316AE08031DDE
:1001D000EB288312F028831283162E088312BE00A8
:1001E000003483162E088312A301B00083162D0855
:1001F0008312AF0002308316AF000130B0008312CB
:100200002D200B138B138B1B022983162F088312AF
:10021000B200B20DB20DB20DF830B2052916C030E1
:100220008B04061133150034640083163C088312D6
:100230008F0083163B0883128E000C100C1C1E29A5
:1002400000340611FF308316BC00CD30BB00831292
:1002500014218316B00183122D2000340C10831654
:100260003C0883128F0083163B0883128E0083168E
:10027000A301A2018312871C5E290C1C4229FF30B6
:10028000A1007E2987183D290F08A3000E08A000B1
:100290000F082302031D442920088316A20083129D
:1002A00023088316A3003B08A2023C08031CA303F7
:1002B000A30200308312A1007E297E290C1C632931
:1002C000FF30A1007E29871C5E290F08A3000E08BD
:1002D000A0000F082302031D652920088316A20031
:1002E000831223088316A3003B08A2023C08031CC8
:1002F000A303A30201308312A1007E2900348316D8
:10030000B10183121D3083163102031C8929831227
:1003100094298312443083163107840080018312AC
:100320008316B10A83128229871101308316B30024
:100330008312B82014308316B40083129720023041
:100340008316B500B401EC30BC007830BB008312DA
:100350002E2121088316B300B31BB0298312B429C0
:1003600083120030A100F2296400EC308316BC0037
:100370007830BB0083122E2121088316B300B31BF3
:10038000C3298312C72983120030A100F2290C303F
:1003900083162302031CCE298312DF2983120B301C
:1003A000831623020319D6298312E2298312B93056
:1003B000831622020318DE298312E22983120130F8
:1003C000A100F229831634080319B503B40383127C
:1003D0008316340835040319EF298312B4298312D4
:1003E0000030A10021088316B000B008031DFA29CF
:1003F0008312842A83128715F4308316BC00483098
:10040000BB0083122E21F6308316BC00BB01831281
:10041000142107308316B3003308B500B50DB50DB0
:10042000FC30B505B4018312FE106400443083161D
:100430003407B60083127E1080308316BA00B701ED
:100440000830B9008312F7308316BC00CC30BB00F3
:1004500083122E2121088316B800B81B312A83127B
:10046000362A83127E140030A100502A87183C2AB5
:1004700083163A08B704831203108316BA0CB90323
:10048000F830BC00BB00831214218316B90803198D
:100490004B2A8312232A8312831637088312A10062
:1004A0008316360884008312210880007E1C5E2A91
:1004B000FE14831635088312A1006B2A8316B40A32
:1004C000B50383128316B5080319682A8312152A07
:1004D00083120030A10021088316B2008312871115
:1004E0008316B3018312B820FE187D2A8316B20842
:1004F000031D7C2A8312812A83120630A1008A2AD6
:10050000842A0030A1008A2A8316B3018312B820FE
:100510000530A10000340710FB308316BC00BB017E
:100520008312142107148316B708031D992A831216
:10053000A22A8312FA308316BC002430BB00831237
:100540001421A92AFF308316BC003830BB00831267
:100550001421003483162E0880390038031DB22A76
:100560008312B82A83128316AE01B0018312C12A06
:10057000013083162E02B000B00DB00DFC30B00576
:100580008312071001308316B70083128B22831663
:10059000B70183128B228316AF08031DD12A831261
:1005A000D82A831201308316B70083128B22DC2AEB
:1005B0008316B70183128B228316B1018312043094
:1005C00083163102031CE62A8312132B8312640064
:1005D00044308316300784000008B2003208B300AC
:1005E0008030B400B5018312083083163502031C35
:1005F000FB2A83120C2B8312831633083405B600B2
:100600003608B70083128B2203108316B40C8312B2
:100610008316B50A8312F42A8316B00A831283164E
:10062000B10A8312DF2A83162E080439B200320879
:10063000B70083128B2283162E080239B2003208CB
:10064000B70083128B2283162E080139B2003208BC
:10065000B70083128B220710F3308316BC001C30C6
:10066000BB0083121421071411308316B4008312C7
:100670009720003401308316B3008312B820323043
:100680008316B4008312972001308316AE002D0824
:10069000AF008312AA2202308316AE002D08AF00ED
:1006A0008312AA2203308316AE002D08AF008312F6
:1006B000AA2204308316AE002D08AF008312AA22AE
:1006C00005308316AE002D08AF008312AA22063033
:1006D0008316AE002D08AF008312AA2207308316BE
:1006E000AE002D08AF008312AA228316B301831235
:1006F000B82000348316AD0183121C3083162D02FE
:10070000031C842B8312972B8312613083162D07D1
:10071000AE0044302D0784000008AF002E0884008E
:100720002F08800083128316AD0A83127D2B0034BC
:100730007F2121088316AD0005302D020319A22B5D
:100740008312A82B8312A1308316AF008312D42BFF
:100750008316AD080319AE2B8312D42B83120230FB
:100760008316AF00AE0183121C3083162E02031CC9
:10077000BB2B8312D42B8312613083162E07840087
:100780000008B00044302E07840000083002031D2A
:10079000CB2B8312D02B8312A4308316AF0083128D
:1007A0008316AE0A8312B42B83162F088312A1007E
:1007B00000348316AD0183121C3083162D02031CF6
:1007C000E32B8312F62B8312443083162D07AE00E1
:1007D00061302D0784000008AF002E0884002F0828
:1007E000800083128316AD0A8312DC2B0034871538
:1007F0003311061501308316B00083122D2001300D
:100800008316AD000530AE008312DA203608A00052
:1008100020080319402C183020020319412C3030D5
:10082000200203194F2C313020020319952C32304D
:1008300020020319B82C333020020319C82C34309D
:1008400020020319EE2C353020020319182D363002
:1008500020020319352D373020020319442D38307A
:1008600020020319562D3930200203196E2D3A301B
:1008700020020319992D3B3020020319E02DF82D99
:10088000F92D8316A801A7012708A800A701A7141E
:100890002808AE002708AD008312F120F92DA13001
:1008A0008316A40083123608B70021210130831675
:1008B000B3008312B82005308316AE0083126400A3
:1008C000EC308316BC007830BB0083122E21210847
:1008D0008316AD002D0A03196F2C8312772C831217
:1008E0008316B3018312B8200030A100872C831631
:1008F000AE0383128316AE080319802C83125F2C7B
:1009000083128316B3018312B8200130A10021089D
:100910008316AB00AB08031D8F2C8312942C83121B
:1009200001308316A4008312F92DA2308316A4008F
:1009300083123608B70021217F2121088316AB00DE
:1009400005302B020319A62C8312AC2C8312A13084
:100950008316A4008312B72C8316AB080319B22C9C
:100960008312B72C831202308316A4008312F92D50
:10097000A3308316A40083123608B7002121831602
:10098000AD0183123A2303308316A4008312F92D9C
:100990008316AD0183121C3083162D02031CD22C4A
:1009A0008312DE2C8312443083162D078400FF301F
:1009B000800083128316AD0A8312CB2CA3308316DA
:1009C000A40083123608B70021218316AD018312DB
:1009D0003A2303308316A4008312F92D0130350227
:1009E000031D172D39088316A9001C30290203188E
:1009F000FB2C8312FF2C83128316A901831244302F
:100A000083162907840000088312A3018316A70018
:100A1000831223088316A8002708A800A701290825
:100A2000A7042808AE002708AD008312F120F92D95
:100A300002303502031D342D3A088316A9008312B3
:100A400039088316AA001C3029020318292D8312A5
:100A50002D2D83128316A901831244308316290792
:100A600084002A0880008312F92D7A23A43083168B
:100A7000A40083123608B700212198232108831689
:100A8000A4008312D923F92D8316A8012408A700F6
:100A90002708A800A701831237088316A70428088F
:100AA000AE002708AD008312F120F92D0130350288
:100AB000031D6D2D39088316A900A908031D622D99
:100AC0008312692D831201308316B3008312B8207C
:100AD0006D2D8316B3018312B820F92D7A23A5302A
:100AE0008316A40083123608B70021218316AC01B7
:100AF0000130B3008312B82032308316B400831261
:100B00009720C4011430C5008030C600EA30C70009
:100B1000FF308316AE002C08AF008312AA22831682
:100B2000B3018312B820D92305308316A4008312A1
:100B3000F92D7A23A4308316A40083123608B70057
:100B400021218316AA01A90183121C3083162902D0
:100B5000031CAC2D8312D02D831244308316290739
:100B600084001C308312A0008316290883122002FF
:100B7000800044308316290784002A088312A000CD
:100B8000A00EA00DE030A005200800048000831610
:100B9000AA0A0730AA0583128316A90A8312A52D73
:100BA0008316AD0183123A2332308316B4008312C8
:100BB0009720982321088316A4008312D923F92DA6
:100BC00001303502031DF72D39088316A900A90845
:100BD000031DEC2D8312F32D831201308316AD001B
:100BE0008312CA20F72D8316AD018312CA20F92D76
:100BF000F92D331D21218711003484011F30830515
:100C00009F308400073080000B138B138B1B052E45
:100C100001308316850083120516CB3083168600BB
:100C2000F2308700813084008017831286018501AD
:100C300087018316B00183122D20061141287528E3
:100C400080288316B3018312B8208316AD01831266
:100C5000CA208316A4018312B6013608B700B50175
:100C6000F723C0308B046400B3123312A91C852E05
:100C7000A910C101C001331C722E0C302B02031DC0
:100C8000712E0B138B138B1B422EAB012D08B8005A
:100C90002C088316A5008312AC01AD01C0308B0473
:100CA00034083802031D702E831625083F3983123D
:100CB000B600831625088312B500B50EB50CB50C29
:100CC0000330B505B314B50803196F2EB3113508F9
:100CD000BF00BF0DBF0DBF0DF830BF05702EB3159F
:100CE0003310852EB31C852E3F082B02031D852E45
:100CF0000B138B138B1B792E2C08B9002D08BA000F
:100D00002E08BB00C0308B04B3150B1DAB2E8330F7
:100D100081000B11B316061C8F2EC00A902EC00145
:100D200007304002031C982E3318982E33143920B4
:100D3000C10A1F304102031CA62EC1013310392005
:100D40002912B2080319A62E0030A62EC20BAB2E14
:100D50001430C2003316B31CB12EB31DB12EF723CD
:100D60003920291EC42EB208031DC42E0618C42E15
:100D7000FF308316BC008230BB008312142183161F
:100D8000B00183122D202912331ED42EC30BD42E72
:100D90006430C300BE080319D42EBE0BD42E8316B4
:0C0DA000AD01AE018312DA20332E630097
:02400E00FD3F74
:041D9C000000020041
:00000001FF
